:10000000F2EF03F01200FFFF04EF04F01200FFFF15
:100018000CEF04F01200FFFFFFFFFFFFFFFFFFFFE1
:10002A000100FC0700006C00000004000000000151
:10003A007C6B1E0E716E0401400E096F200E0A6F52
:10004A00040E0B6F880E086F0401200E0E6F040E4B
:10005A000F6F400E0C6F1200550EA76EAA0EA76EF8
:10006A00A68212000401226B010E236F1200000106
:10007A007A6B0401215100017A5D20E27AC000F016
:10008A00016A026A040122510024F36E23510120FD
:10009A00F46E24510220F86EF4CFF7FFF3CFF6FF87
:1000AA000800F5CF7BF000017A51EA6A250FE96E64
:1000BA00040EEA227BC0EFFF7A2BDBD7F86A120024
:1000CA00F00E04012217840EA66E00017A6B040159
:1000DA00215100017A5D26E27A51EA6A250FE96E1A
:1000EA00040EEA22EFCF03F07AC000F0016A026A36
:1000FA00040122510024F36E23510120F46E24518D
:10010A000220F86EF4CFF7FFF3CFF6FF03C0F5FF36
:10011A000C000F0E00017A150F0801E19DDF0001A6
:10012A007A2BD5D71200940EA66E00017A6B0401C1
:10013A00215100017A5D1EE27A51006E016A060EB3
:10014A00D89000360136E804FBE1026A01BE026873
:10015A00040122510024F36E23510120F46E24512C
:10016A000220F86EF4CFF7FFF3CFF6FF75DF000138
:10017A007A2BDDD7F86A1200A66A00017A6B0401AD
:10018A00215100017A5D10E20401225100017A2511
:10019A00A96EA6807A51EA6A250FE96E040EEA2250
:1001AA00A8CFEFFF7A2BEBD7120000017A6B04017C
:1001BA00215100017A5D15E20401225100017A25DC
:1001CA00A96E7A51EA6A250FE96E040EEA22EF5007
:1001DA00A86E040EA66E40DFA6B2FED700017A2BE7
:1001EA00E6D71200C40EA66E00017A6B04012151F3
:1001FA0000017A5D21E27A51EA6A250FE96E040E5E
:10020A00EA22EFCF03F07AC000F0016A026A040121
:10021A0022510024F36E23510120F46E245102204E
:10022A00F86EF4CFF7FFF3CFF6FF03C0F5FF0C002B
:10023A0013DF00017A2BDAD7F86A1200060E0001E2
:10024A007F5D03E36D50020B01E074D000017C0571
:10025A0011E104010CBF0DD00401400E096F400EDC
:10026A00040108170401087D880E0401081300011F
:10027A007C6B60D0040108BF5DD000017A6B040179
:10028A002051320A45E0CD0A34E0F80A2DE0020A8C
:10029A0026E0010A1FE0070A18E0010A11E0030A32
:1002AA000AE0070A08E0060A01E033D0DBDE0001B3
:1002BA00040E7A6F2FD0DBDE050E00017A272AD0D2
:1002CA00FFDE0001010E7A6F25D02DDF0001010E3D
:1002DA007A6F20D051DF050E00017A271BD065DF27
:1002EA000001010E7A6F16D07DDF0001010E7A6FD0
:1002FA0011D06D9600017D6B7E6B00017D07000EAB
:10030A007E5B00017D517E1101E0F7D7FF0002D02C
:10031A0001D000D00001010E7C6F00017A510AE081
:10032A007AC00DF4400E04010C1704010C7D880EEE
:10033A0004010C1312006C5002E0000E01D0010EF1
:10034A0000090BE0040100513C0BE842E8420D08A9
:10035A0002E1BBEF01F0C4EF01F06C5002E0000EC5
:10036A0001D0010E040901E019D812000001606BE6
:10037A00616B666B676B99EC02F046EF02F0020E56
:10038A000001605D09E15CD8040100BD02D0C80E1D
:10039A0001D0880E006F12008BEF02F0040E0001EC
:1003AA007F5D09E112C46EFF6E50000802E2050E7D
:1003BA0001D0030E7F6F0001600509E10AD804012C
:1003CA0004BD02D0C80E01D0880E046F12008BEF54
:1003DA0002F00001080E665D000E675903E266C06E
:1003EA0069F002D0080E696F69C005F46951006EA0
:1003FA00016A0050665F0150675B180E646F040E55
:10040A00656F69511CE0000180A307D062C0F6FF46
:10041A0063C0F7FF0800F55005D062C0E9FF63C06A
:10042A00EAFFEF5064C0E9FF65C0EAFFEF6E000122
:10043A00622B000E6323642B65236907E2D712003F
:10044A0001C46AF000016A516625666F000E6721D1
:10045A00676F180E626F040E636F6A5111E062C013
:10046A00E9FF63C0EAFFEF5064C0E9FF65C0EAFF35
:10047A00EF6E642B000E6523622B63236A07EDD7A8
:10048A001200000161510BE10401080E016F100E08
:10049A00026F040E036F840E006F040123D004015F
:1004AA0010AF22D0000166510401165D00016751A8
:1004BA000401175904E216C466F017C467F089DF0D
:1004CA000001010E606F0401080E016F100E026F29
:1004DA00040E036F800E006F0401180E066F040EDF
:1004EA00076FC80E046F10D00001020E606F04017E
:1004FA00056BC80E046F0401080E016F180E026F17
:10050A00040E036FC80E006F6D9812000001606B35
:10051A000401080E016F100E026F040E036F880E9D
:10052A00006F0401046B120004011051600BE842D1
:10053A00E842E842E842E842000901E012001151AB
:10054A00080A39E0010A35E00F0A0AE0030A01E065
:10055A0012000001010E616F0001040E7F6F12008C
:10056A000001010E616F0401130507E10001AE0EDF
:10057A00626F070E636F120E13D0020E135D07E14E
:10058A000001C00E626F070E636F200E09D0030EC2
:10059A00135D0AE10001E00E626F070E636F040E3D
:1005AA000001666F676B02D00001616B00018083F6
:1005BA001200EEEF02F00001010E616F0001810EE0
:1005CA00626F000E636F000180930001010E666F77
:1005DA0012000001010E616F12C481F00401125170
:1005EA0004E10001050E7F6F12000001060E7F6F05
:1005FA001CEF00F0080E6D6E6DBAFED7686A110E18
:10060A00696E0001020E7F6F12006850040B06E04B
:10061A006950040B03E06D92699468946850010B69
:10062A0004E06950010B01E027D86850100B09E07B
:10063A006950100B06E0698468986D82A08A0300ED
:10064A00A19A6850200B09E06950200B06E070A0BF
:10065A0003D08BEC02F07090689A030E00017F5D64
:10066A0001E209D06850080B06E06950080B03E064
:10067A00A0EC01F068961200686A7B0E696E6E6AD9
:10068A00160E706E68A602D06896FCD76D988BEC31
:10069A0002F00001816B0001030E7F6F12002A0E27
:1006AA00F66E000EF76E000EF86E00010900F550A6
:1006BA00756F0900F550766F03E1756701D03DD07B
:1006CA000900F550706F0900F550716F0900F55077
:1006DA00726F09000900F550E96E0900F550EA6EDB
:1006EA00090009000900F550736F0900F550746F8D
:1006FA0009000900F6CF77F0F7CF78F0F8CF79F054
:10070A0070C0F6FF71C0F7FF72C0F8FF00017353A3
:10071A0002E1745307E00900F550EE6E7307F8E240
:10072A007407F9D777C0F6FF78C0F7FF79C0F8FFEA
:10073A0000017507000E765BBFD71200C1CF83F0A8
:10074A000F0EC1127F0EF16E0001846B9384949098
:10075A008280CF6ACE6A9E90310ECD6E81A404D07B
:10076A0083C0C1FF00EF04F0140E6F6EFFEC02F0BD
:10077A000AEC03F023EC01F09EA012D09E90000137
:10078A00842B0F0E0001845D0BE30001846B825001
:10079A00010B010A010BF36EFE0E8214F310826E36
:1007AA00E7D712001201000200000008D8040B006B
:1007BA000000000000010902200001010080320946
:1007CA0004000002000000000705010240000007C3
:1007DA000581024000000403090413EE00F023EE31
:1007EA0000F0F86A059C54EC03F0A3EC03F0FDD783
:1007FA0012006B695DEA9CEF14F01200FFFFD1EF63
:10080A0012F01200FFFFFFFFFFFFFFFFFFFF47EF9E
:10081A0013F01200FFFFFFFFFFFFFFFFFFFFFFFFC5
:10082A00010062290000600000007C000000EFDA8D
:10083A000001010EF56FF66FF76F330EEF6FE66A80
:10084A00CADAE5520001F069F1691200D9CFE6FF70
:10085A00E1CFD9FF070EE126060E0201F55D03E39B
:10086A006D50020B0AE00001F007000EF15B000177
:10087A00F051F11101E1FF0017D10001F551040A0D
:10088A0001E1F9D0070A01E1CBD0010A17E0030A16
:10089A0001E006D18280010EE66EF20EE66E000ECF
:1008AA00E66E8EEC0EF0E552E552E552000905E0DF
:1008BA00F2C0F3F00001020EF56FF6D00201D15139
:1008CA0001E0ADD0FF0E0001F35D07E190DA000907
:1008DA0003E00001010EF56FA2D0800E0001F35D66
:1008EA0006E10001F46B0001030EF56F98D0810E4A
:1008FA000001F35D1FE18290000EE66E020EE66EC5
:10090A00000EE66E010EE66ECADBE552E552E552CE
:10091A00E552E76E060EE7CFDBFF060EDB0405E1C4
:10092A0082800001040EF56F04D082800001010E5E
:10093A00F56F75D0800E0001F35D55E2030E0001DC
:10094A00F315E76E010EE7CFDBFF0C0E0001F3157E
:10095A00E840E8403F0BE76E020EE7CFDBFF020EEE
:10096A00DB50030805E1020EF36E020EF3CFDBFF44
:10097A00300E0001F315E8380F0B010FE76E030E76
:10098A00E7CFDBFF030EDB50030805E1040EF36E2D
:10099A00030EF3CFDBFF060E146E400E0001F315B3
:1009AA0014C0E7FFE75204E0E8427F0BE706FCE1E8
:1009BA00E76E040EE7CFDBFF040EDBCFE6FF020E85
:1009CA00DBCFE6FF010EDBCFE6FF030EDBCFE6FF50
:1009DA00C7D8E552E552E552E552000903E00001A5
:1009EA00010EF56F1CD0DF6A0E0EDF5C15E2DF50D8
:1009FA00EA6ACE0FE96E000EEA22EF500001F35DBB
:100A0A0009E18290DFCFE6FF150EE66EB8EC0AF038
:100A1A00E552E552DF2AE8D70001010EF56F44D00E
:100A2A008290000EE66E020EE66E000EE66E010E73
:100A3A00E66E5EDAE552E552E552E552E76E050EDC
:100A4A00E7CFDBFF050EDB5015E0050EDB040EE1F8
:100A5A00000EE66E020EE66E000EE66E010EE66E01
:100A6A0007EC0CF0E552E552E552E5520001010EA1
:100A7A00F56F828019D08290000EE66E020EE66E45
:100A8A00000EE66E010EE66EC2DAE552E552E55256
:100A9A00E552000904E00001010EF56F828004D0DE
:100AAA000001010EF56F00D0D9CFE1FFE552E7CF83
:100ABA00D9FF1200C6EC09F08290EFC081FF140E34
:100ACA00E66EF8D9E552FE0EDB500B0DF3CFECF0D3
:100ADA000001F350E0EC09F0EECFEDF0EDCFEEF0CF
:100AEA00F328E0EC09F0EECFE2F0EDCFE3F0020EEE
:100AFA00F324E0EC09F0EECFE4F0EDCFE5F0030EDD
:100B0A00EC27DE6BDF6BE06BE16BDD6BF28C32ECBA
:100B1A000AF0BD6A050EBD6E9E6AF28EDDA5FED78D
:100B2A00F29E330E816EDDB303D01DEC0AF016D0AF
:100B3A00EA51E65DEB51E7590BE2E851E91104E0AD
:100B4A00E807000EE95B04D01DEC0AF0EA6BEB6BD8
:100B5A00EA51E65DE66FEB51E759E76FCBEF09F033
:100B6A00C6EC09F0410EE1263B0EDB6A360EDB6A63
:100B7A00030EF36E370EF3CFDBFF020EF36E380E61
:100B8A00F3CFDBFF010EF36E390EF3CFDBFFFD0E61
:100B9A00DBA003D03C0EDB6A05D0030EF36E3C0EDD
:100BAA00F3CFDBFFFD0EDBA202D0040E01D0030E51
:100BBA00F36E3D0EF3CFDBFF0001F651060A01E1A9
:100BCA00EDD0030A01E1DCD0010A01E1C3D0070A32
:100BDA0001E1B4D0010A6DE0030A01E0E6D00201A6
:100BEA00C86B180EC85D05E2C0DBEE6AED6AC82B59
:100BFA00F8D7400EDB6AFE0EDB50F36E400E75EC42
:100C0A000AF052E23C0EDB50E76E3E0EE7CFDBFF06
:100C1A003D0EDB50F36E3E0E75EC0AF042E2D950FF
:100C2A00360F146EDACF15F03E0EDB500F01142486
:100C3A00E96E000EDA20EA6EEF50E66EBDD8E55294
:100C4A00FC0EDB50020818E13F0EDB6ADB5001089C
:100C5A0025E33F0EDBCFE6FFBED8E5525EDBD8A028
:100C6A0002D062EC0AF0D9CF14F0DACF15F049ECD1
:100C7A000AF03F0EDB2AEAD73F0EDB6AFC0EDB5096
:100C8A00030805E0FC0EDBCFE6FFA5D8E55245DBFD
:100C9A00D8A002D062EC0AF049EC0AF03E0EDB2A38
:100CAA00B7D7400EDB2AA7D70201C86B180EC96F47
:100CBA0072D0FD0EDBA00CD0520EF36E300EF3CFC5
:100CCA00DBFF470EF36E310EF3CFDBFF420E0BD084
:100CDA005F0EF36E300EF3CFDBFF5F0EF36E310E55
:100CEA00F3CFDBFF5F0EF36E320EF3CFDBFFFD0EA9
:100CFA00DBA202D0570E01D05F0EF36E330EF3CF94
:100D0A00DBFFFC0EDB50020802E1320E05D0EFA930
:100D1A0002D0310E01D0300EF36E340EF3CFDBFF6A
:100D2A003A0EF36E350EF3CFDBFF0201D15106E125
:100D3A000201D950300FB0DB0001F62B0201D1516C
:100D4A0036E102015B0ED26F290ED36F0201060E45
:100D5A0060DB21D0D9CF14F0DACF15F0020105DB20
:100D6A00EECFE6FFEFCFE6FF74D8E552E552000971
:100D7A0002E00201C82B0201C951C85D18E30BD079
:100D8A000201D15114E10201580ED26F290ED36F1C
:100D9A000201020E3EDB0001F62B09D0010EF66FAE
:100DAA00F36E3B0EF3CFDBFF02D0010EF66F3B0E64
:100DBA00DB50D9CFE1FFEAD2E4DAFE0EDBA003D0A2
:100DCA000001EF8D02D00001EF9DDBA202D0EF8F70
:100DDA0001D0EF9FDBD2D5DAFE0EDB5004E1000131
:100DEA00EF81EF9903D00001EF91EF89CFD27DDB3C
:100DFA000201D15109E10201500ED26F290ED36FBF
:100E0A000201070E06DBDF6EDF50E552BFD2806AB1
:100E1A00826A330E816E92680C0E936EFE0E946E89
:100E2A00D06A400EF26E800EF16E050E9D6ECD6A8E
:100E3A00BD6ECA6E0F0EBA6E1200110ECB6E090E7F
:100E4A00BB6E040ECA6E0F0EBA6E0001DC6B949272
:100E5A00120097DA090EE126DF6AFE0EDB50E76E12
:100E6A00070EE7CFDBFF20DB010E21DB020E02DBE0
:100E7A00030EE7CFDBFFFD0EDBCF14F0FE0EDBCF58
:100E8A0015F00001156A070E14C0DBFF0DDB040E16
:100E9A000EDB050EEFDA060EE7CFDBFF0201D151BA
:100EAA0005E10201D950010FF7DADF6EDF50D9CF21
:100EBA00E1FF6CD266DA020EE126DF6AFE0EDB5033
:100ECA00DF5C13E2010EDB6ADF50146E156AD890FC
:100EDA00155004E6FA0E145C000E155804E2DF2AD7
:100EEA00DF06DF2AF1D7DF2AE9D7D9CFE1FF4ED2D1
:100EFA00FCDA0001F45107E1010EF46F0201CA6B3A
:100F0A00CB6BCC6BCD6B010EE66EF20EE66E000E6D
:100F1A00E66E8EEC0EF0E552E552E55200096AE003
:100F2A000201CC6BCD6BC80ECA5D000ECB590BE229
:100F3A00FD0EDB50CA250F01E96EFE0EDB500201E1
:100F4A00CB210F010FD0CAC214F0CBC215F0C80EC4
:100F5A00145E000E155AFB0EDB501424E96EFC0ECB
:100F6A00DB501520EA6EF2C0EFFF0201CA2B000E19
:100F7A00CB23900ECA5D010ECB5902E3020E43D079
:100F8A00080ECA5D000ECB593FE3010EBFD9EF50E0
:100F9A00500805E0010EBAD9EF50600806E10C0EC0
:100FAA00CA5D000ECB5930E323D0040EAFD9EFCF80
:100FBA0018F0060EABD9EF501824166E176A000EF9
:100FCA001722040E066E076A16C00BF017C00CF043
:100FDA0041EC14F004C014F005C015F0080E1426F4
:100FEA00000E152202011450CA5D1550CB590CE3AC
:100FFA00010E09D00201CC2B000ECD23CC1D04E139
:10100A00CD1D02E1020EDF6EDF50E552BFD16DDA6F
:10101A000001F751030A2EE0010A17E0030A3AE138
:10102A00040E066E076A04C10BF005C10CF041EC10
:10103A0014F004C0CEF205C0CFF2080E0201CE278A
:10104A00000ECF230001F72B27D00201D15112E164
:10105A000201C80ED880CE55000ECF5504E3EFD951
:10106A0032DAF76F07D0EBD90201C80ED66FBDD9B5
:10107A000001F72B0201D1510FE10201C80ECE5F28
:10108A00000ECF5BFB0EDBCFD2F2FC0EDBCFD3F22E
:10109A001ADA01D0010EF76FDF50E55277D171D914
:1010AA000E0EE126040EDB6A070EDB6A050EDB680C
:1010BA00040EF36E080EF3CFDBFFDE68DD68020E66
:1010CA00DB6A030EDB6A0B0EDB6A0C0EDB6A0D0EA3
:1010DA00DB6AFFD9EE6AED6A020E18D96D0EEE6E62
:1010EA00ED6A040E13D9EE6AED6A060E0FD9EE6A9E
:1010FA00ED6A010EE66E6FDEE552EFC081FFBD6A52
:10110A00050EBD6EAAD9010ECA6ECC6A4F0ECB6E01
:10111A00050ECA6E9E6A070EDB5001E0DFD09EB252
:10112A0015D09EA4FCD79EA003D0DE68DD680AD045
:10113A00BF50166E176A176E166ABE5087D914C04A
:10114A00DEFFDD6E8AD99E949E90E9D79E92CF509B
:10115A00166E176A176E166ACE5078D9020E14C028
:10116A00DBFF030E15C0DBFF9EA004D0020EDB6876
:10117A00030EDB68DECF14F0DDCF15F0780E145CB9
:10118A00020E155811E2020EDBCF16F0030EDBCF6A
:10119A0017F0780E165C020E175806E2010EF36E6F
:1011AA00060EF3CFDBFF02D0060EDB6A050EDB501C
:1011BA00FF081DE1060EDB0401E182D0D9500B0FB6
:1011CA00E96EDACFEAFFEE2A000EEE22EE22D950BD
:1011DA000B0FE96EDACFEAFFE868EE189CE1E868DF
:1011EA00EE1899E1050EEE1896E1020E62D0050E90
:1011FA00DB50F36E060EDB50F35C1EE1090EDB2AB0
:10120A000A0E01E3DB2AD950090FE96EDACFEAFFA9
:10121A00FF0EEE1801E07FD7080EED1801E07BD72C
:10122A00010EF36E070EF3CFDBFFB4D802E2E3D868
:10123A0001D0CBD8F5D86FD7ADD802E2DCD801D02F
:10124A00C4D8EED8080EDB50146E156AC70E1418EF
:10125A0035E1155033E19ED824E3FB0EDBCF16F0BF
:10126A00FC0EDBCF17F0080EDB509C0F020D165058
:10127A00F324E96E1750F420EA6EEECF14F0EFCFA4
:10128A0015F0000E145C020E15580BE2020E146ED5
:10129A00080EDBCFE7FF1450E75E080EE7CFDBFF4F
:1012AA00DAD778D805E2C70EF36E080EF3CFDBFF64
:1012BA00010EF36E070EF3CFDBFF2DD7080EDB2AE4
:1012CA00010EF36E090EF3CFDBFF0A0EDB6A060E80
:1012DA00DB50E76E050EE7CFDBFF1DD7080EDB50AC
:1012EA00FD0FFE0BE842E66E040E10D8E552E750F9
:1012FA00EE6EED6A330E816E070EDB50E76E040E5A
:10130A00E7CFDBFFDB50D9CFE1FF40D0E76EE1D872
:10131A00E750E926000EEA221200FB0EDBCFE6FFB9
:10132A00FE0EDB04E552E724E66E5FEC05F0E552BB
:10133A003F0EDB500C0DF3CF14F03E0EDB50030DC5
:10134A00F35014240201C86F020EC8258BD800017D
:10135A00E051EE26E151ED220201C82983D80001AD
:10136A00E651EE26E751ED221200C85137EF0AF096
:10137A00146E0C6E070EDBCF07F08EEC14F0080E1D
:10138A001200D9CFE6FFE1CFD9FF1200E552E7CF2D
:10139A00D9FF1200640EF36E080E75EF0AF003C04F
:1013AA00DBFF0A0E146E0C6E080EDBCF07F08EEC14
:1013BA0014F0080E9ED0E96EEA6AD890E936EA3649
:1013CA00600EE926000EEA221200FB0EDBCF14F0B3
:1013DA00FC0EDBCF15F0080EDB509C0F020D1450EB
:1013EA00F324E96E1550F42012000201D76B0201B2
:1013FA00010ED16F1200080E156ADB34FE0B15368A
:10140A00146EFD0EDB501424E96EFE0EDB5015201F
:10141A001200D66F0201010ED76F0201D16F1200BE
:10142A00EA6E090EDBCFEEFF0A0EDBCFEDFF1200EC
:10143A00E86BE96BE66BE76BE06BE16B1200FD0EA4
:10144A00DBCFD2F2FE0EDBCFD3F21200000116245C
:10145A00146E000E1720156E1200CD90CF6ACE6A58
:10146A00CD801200020DD950F324E96EDA50F4202F
:10147A00EA6E1200E7CFDBFF0A0E7ADF03C0DBFF5A
:10148A00DB50300FE76E120002016FDF0001E851F6
:10149A00EE26E951ED221200D26FDACFD3F2020121
:1014AA00060ED66FFAEF09F0640E62DF22D0E7CF9C
:1014BA00DBFF640E5DDFD4EF09F0020156DFEE2A8E
:1014CA00000EEF221200CEC2D6F28FDFDF6E0001CD
:1014DA001200FD0EDBCFE9FFFE0EDBCFEAFF1200A2
:1014EA00DBCFF4FFF350F45C12004BDFE652DF6A05
:1014FA00120007C0DBFFDB50300FE76E12006DDA17
:10150A00F2A4FED7B5DA03E02A0EBB6E01D0BB6A9D
:10151A0069D24DDBDF5000080AE2FE0EDBAE03D0D3
:10152A00010EE66E01D0E66AEADF8DDAF3D7E552FC
:10153A0059D253DAE652080EDF6EDF50000811E284
:10154A00FE0EDBAE06D0010EE66ED9DFE552E66A84
:10155A0005D0E66AD4DFE552010EE66ED0DF73DA13
:10156A00ECD7E5523FD239DA9492530ECB6EC40EC1
:10157A00D56E590ED66EF2942A0EBB6E070EE66E23
:10158A00F80EBADA080EE66E950EB6DA040EE66EB4
:10159A00300EB2DAFE0EDBCFE6FFCBDFE552FD0EF0
:1015AA00DBCFE6FFC6DFE552E66AA9DFE5529482A1
:1015BA0019D213DAF2A4FED75BDA03E02A0EBB6E65
:1015CA0001D0BB6A0FD2F3DADF50000811E2FE0E37
:1015DA00DBAE06D0E66AEDDFE552010EE66E05D017
:1015EA00010EE66EE6DFE552E66AE3DF2CDAECD7B7
:1015FA00E552F8D1F2D99492530ECB6EC50ED56E40
:10160A00FA0ED66EF294BB6A030EE66EC00EE66E52
:10161A00DADFE552E552FE0EDB50080DFE0EF3CF7F
:10162A00DBFF050EE66EFE0E78DAFD0EDB50040DCA
:10163A00FD0EF3CFDBFF060EE66EFD0E6EDAE66AEE
:10164A00B8DFE5529482CED1C8D9130EE126FC0E3A
:10165A00DBCFF6FFFD0EDBCFF7FFFE0EDBCFF8FF89
:10166A000900030EC9DA040EF5CFDBFF010EC0DA5A
:10167A000D0EC2DA0E0EF5CFDBFFB2DAED1001E085
:10168A00ADD0020EE76E4FDAE7501626000E17228B
:10169A00186AD890163617361836B2DA1624F36E48
:1016AA00EE501720F46EEE501820B2DAF5CF14F08F
:1016BA000800F5CF15F0830E1502F3CF15F01402CA
:1016CA00F3CF14F0F4501526090EF3CFDBFF0A0E00
:1016DA0015C0DBFFB50E146E156A6FDA2BDA090E28
:1016EA00DBCF14F00A0EFDD968DA0B0E06C0DBFF59
:1016FA000C0E07C0DBFFBB6A030EE76E3FD9050E6F
:10170A007BDA060EF5CFDBFF040E72DA070E74DA07
:10171A00080EF5CFDBFF94929EA2FED79E920B0E87
:10172A00DB50BB6E030EDBCF14F0040EDBCF15F0DB
:10173A00050E1424DF6E5AD92ADAA7D915E230D950
:10174A0039D909E29EA2FED7010EDB06020E01E29A
:10175A00DB069E92F5D7BB5004E10B0EDB50BB6E45
:10176A0001D0BB6ADF2AE7D7DED911DA41EC14F0DF
:10177A0016500424146E17500520156E050E1424F5
:10178A00DF6E34D9070EDBCF1BF0080EDBCF1CF05F
:10179A00050EDB501B24196E060EDB501C201A6E38
:1017AA00B8D919C00BF01AC00CF06FD915E2F8D8E5
:1017BA0001D909E29EA2FED7010EDB06020E01E262
:1017CA00DB069E92F5D7BB5004E10B0EDB50BB6ED5
:1017DA0001D0BB6ADF2AD5D7948211D001DA06E19B
:1017EA00600EED1803E1BCD9BEDE07D0F9D907E1D6
:1017FA00500EED1804E1B4D9FDDEE552E552D9CF19
:10180A00E1FFF0D0EAD8110EE126DDD90B0EEECFBA
:10181A00DBFF0C0EEDCFDBFFE7D9ED1001E09AD02C
:10182A00020EB7D8EECF14F0EFCF15F0830E1502E3
:10183A00F3CF15F01402F4501526070EF3CFDBFF91
:10184A00080E15C0DBFFB50E146E156AC3D9070E54
:10185A0006C0DBFF080E07C0DBFF070EDBCF14F064
:10186A00080E3FD9B7D966D9BB6A040E92D8030EBF
:10187A00EECFDBFF040EEDCFDBFF060E8AD8050E96
:10188A00EECFDBFF060EEDCFDBFF94929EA2FED7D2
:10189A009E92090EDB50BB6E82D941EC14F005C052
:1018AA0015F0040E0424DF6EDFCF14F078D9ADD81A
:1018BA001BE2640EDF5C02E2F5D801D0B5D821D96B
:1018CA0079D809E29EA2FED7010EDB06020E01E2DA
:1018DA00DB069E92F5D7BB5004E1090EDB50BB6EC6
:1018EA0001D0BB6ADF2AE0D7040EDF6EDFCF14F027
:1018FA00050EDBCF19F0060EDBCF1AF0030EDB5014
:10190A001924176E040EDB501A20186E02D917C05C
:10191A000BF018C00CF079D81BE2640EDF5C02E20F
:10192A00C1D801D081D8EDD845D809E29EA2FED708
:10193A00010EDB06020E01E2DB069E92F5D7BB50D2
:10194A0004E1090EDB50BB6E01D0BB6ADF2ACED799
:10195A00948211D049D906E1600EED1803E10BD942
:10196A0002DE07D041D907E1500EED1804E103D990
:10197A0041DEE552E552D9CFE1FF34D0DBCF14F096
:10198A00040EDBCF15F0E7501426000E1522A6EF41
:10199A000DF0E76E18D9E750E926000EEA22120088
:1019AA00DFCF14F0156ACDD8010E26D9020EF5CF75
:1019BA00DBFF1200D950010FE96EDACFEAFF000E01
:1019CA00D880EE54000EED541200DBCF07F014C09D
:1019DA000BF015C00CF078EF14F0D9CFE6FFE1CF89
:1019EA00D9FF1200E552E7CFD9FF1200DFCF14F07A
:1019FA00050EE76E030EDBCF17F0040EDBCF18F0EF
:101A0A00E7501726000E1822120041EC14F004C009
:101A1A0015F005C016F0040E1526000E16221550F4
:101A2A00145C000E16541200FB0EDBCF14F0FC0EF1
:101A3A00DBCF15F0640EDF5C020D1450F324E96E5F
:101A4A001550F4201200E552FE0EDB50020DFE0E78
:101A5A00F3CFDBFFDF061200110ECED8120EF5CF40
:101A6A00DBFF110EDBCFE6FF0F0EDBCFE6FF120026
:101A7A00D650146E156AA60E145E000E155A14502E
:101A8A00D66EF294FE0EDB50120041EC14F01750A1
:101A9A000424156E18500520166E1550145C000E9D
:101AAA0016541200156ADF34FE0B1536146EFD0E3D
:101ABA00DB501424E96EFE0EDB50152012000F0EC7
:101ACA00EECFDBFF100EEDCFDBFF0F0EDBCFE6FF15
:101ADA000D0EDBCFE6FF1200E96EDACFEAFFEE5019
:101AEA001200DBCF15F01406000E155A1450CB6EF7
:101AFA00020E146E156A1200E66E0BDDE552E5520F
:101B0A001200EA6E010EEECFDBFF020EEDCFDBFF15
:101B1A001200020E066E076A1200DBCFE6FF53DDE3
:101B2A00E552E5521200030EDBCF16F0040EDBCFAE
:101B3A0017F01200090E06C0DBFF0A0E07C0DBFF12
:101B4A001200166AD89014361536163659D8142447
:101B5A00F36EEE501520F46EEE5016200DEF0EF0D7
:101B6A00050E46D80F0E48D8100EF5CFDBFF060E2D
:101B7A003FD831EF0DF0080E0CDF0D0EEECFDBFF74
:101B8A000E0EEDCFDBFF0A0E04DF64EF0DF0C1DFAE
:101B9A00050EDBCF0BF0060EDBCF0CF01200B9DF1F
:101BAA00030EDBCF0BF0040EDBCF0CF0120015DFB7
:101BBA00E652FD0EDB50DF6E1200090EDBCF06F097
:101BCA000A0EEAEF0CF0FD0EDBCFE9FFFE0EDBCFCB
:101BDA00EAFF1200070EDBCF06F0080EEAEF0CF060
:101BEA00D9500D0F71EF0DF0D9500B0F71EF0DF0A9
:101BFA00E76E030EC3EF0CF0F5CFDBFF0A0012000D
:101C0A00D950FC0FE96EFF0EDA20EA6EEE50120090
:101C1A00F86EF4CFF7FFF3CFF6FF090012000401C4
:101C2A0020511F0B010801E012002051600BE8420D
:101C3A00E842E842E842E842010801E01200245181
:101C4A0003E0240501E012002151230A39E0010AC8
:101C5A0033E0030A25E0010A1CE0240A31E0070AFE
:101C6A002FE0010A2DE0030A0EE0010A01E012004A
:101C7A004ED90001E30EFA6F020EFB6F0201F693D2
:101C8A000001080E17D043D90001E30EFC6F020EC3
:101C9A0005D03DD90001D80EFC6F020EFD6F12006F
:101CAA0036D90001D80EFA6F020EFB6F0201F693C5
:101CBA000001070EFE6F12002AD922C4DFF21200B9
:101CCA0012000201D86BC20ED96F010EDA6FDB6BFC
:101CDA00DC6BDD6B080EDE6FD16BD06B1A0E726E89
:101CEA001E0E736E0401000E166F050E176F400E5E
:101CFA00146F0401196F080E1A6F050E1B6F880EF8
:101D0A00186F0401480E1E6F050E1F6F400E1C6FE0
:101D1A001200D9CFE6FFE1CFD9FF0201D06B04014F
:101D2A0018BF30D0FC0EDBCF14F01951D8801454F0
:101D3A0003E2FC0E19C4DBFF0201D06BFC0EDB5080
:101D4A00D05D19E2D051EA6A080FE96E050EEA225F
:101D5A00EF50E66ED051E76EFD0EDBCFE9FFFE0EC7
:101D6A00DBCFEAFFE750E926000EEA22E552E75008
:101D7A00EF6ED02BE3D70401400E196F1817187DA8
:101D8A00880E18130201D051E552E7CFD9FF12008D
:101D9A00ACD80201D15114E1DF6AB2D802E1155080
:101DAA000BE0FD0EDBCFE9FFDB2AFE0EDBCFEAFFFD
:101DBA0001E3DB2AEF50F1E175D8D76B010ED16F41
:101DCA009AD093D80201D15115E1DF6A99D802E17C
:101DDA0015500CE0FD0EDBCFF6FFDB2AFE0EDBCF43
:101DEA00F7FF01E3DB2A0800F550F0E15BD8010EAA
:101DFA00D76FD16F80D079D804011CBF52D0030E9F
:101E0A000201D15D01E1D16BD1514BE0020ED15DEE
:101E1A0003E104011D6B3CD0D1053DE1400E146E77
:101E2A00156AD651145C000E155803E2400EDF6E97
:101E3A0002D0D6C2DFFFDFCF1DF4DF50D65DD66FEA
:101E4A00480ED46F050ED56FD7050AE1DF5011E0B1
:101E5A00D2C2F6FFD3C2F7FF0800F5503AD8F6D738
:101E6A00DF5007E0D2C2E9FFD3C2EAFFEF5031D810
:101E7A00F7D70201D6510FE104011D51146E156AFC
:101E8A00400E141805E1155003E10201020E02D0BA
:101E9A000201030ED16F400E04011C171C7D880E2F
:101EAA001C1329D0DF50146E156AD950FD0FE96E44
:101EBA00FF0EDA20EA6E1450EE5E1550ED5AFD0E52
:101ECA00DBCFD2F2FE0EDBCFD3F2DFCFD6F20201A6
:101EDA001200D4C2E9FFD5C2EAFFEF6ED42B000E7E
:101EEA00D523D22BD323DF061200D9CFE6FFE1CFC9
:101EFA00D9FFE6521200E552E552E7CFD9FF1200A8
:101F0A00DF2ADF50146E156AFF0E14181200000142
:101F1A00030EF96F12006C5002E0000E01D0010EA0
:101F2A0000090BE0040100513C0BE842E8420D08AD
:101F3A0002E1ABEF0FF0E0EF0FF06C5002E0000EA1
:101F4A0001D0010E040901E045D81200D9CFE6FFFD
:101F5A00E1CFD9FFE6520001F86BF96BFE6BFF6B1C
:101F6A00D8EC10F0DF6ADF50146E156A010E145CAB
:101F7A00000E15581AE20001F95117E1F76ADF3429
:101F8A00FE0BF736F66EE10EF626270EF72209004B
:101F9A00F5CF14F00800F5CF15F004D015C0FAFFFC
:101FAA001450F96EFBDFDF2ADED790D8E552E552EE
:101FBA00E7CFD9FF1200020E0001F85D09E162D8ED
:101FCA00040100BD02D0C80E01D0880E006F1200B5
:101FDA00A4EF10F0040E0201F55D09E122C46EFFC0
:101FEA006E50000802E2050E01D0030EF56F0001E3
:101FFA00F80509E10AD8040104BD02D0C80E01D0CF
:10200A00880E046F1200A4EF10F0B8D80001080E71
:10201A00FE5D000EFF5905E2FEC0DEFFFFC0DDFFD8
:10202A0003D0080EDE6EDD6A040104930491010EEA
:10203A00DB500413DFCF05F4000EDB500001FE5F16
:10204A00010EDB50FF5B280EFC6F040EFD6F0201D0
:10205A00F6A30CD08CD815E0FAC0F6FFFBC0F7FF48
:10206A000800F55074D8F6E2DB06F4D780D809E008
:10207A00FAC0E9FFFBC0EAFFEF5069D8F7E2DB06D6
:10208A00F5D783D07BD8030E04010015E76E010E45
:10209A00E7CFDBFF01C4DFFFDE500001FE27DD5082
:1020AA00FF23280EFA6F040EFB6F61D80EE0FAC008
:1020BA00E9FFFBC0EAFFEF50FCC0E9FFFDC0EAFF01
:1020CA00EF6E69D8F2E2DB06F0D75FD00001F95172
:1020DA0005E145D8840E006F04011DD0040120AF2C
:1020EA001CD00001FE510401265D0001FF510401CC
:1020FA00275904E226C4FEF027C4FFF086DF000158
:10210A00010EF86F2CD8800E006F0401280E066F9E
:10211A00040E076FC80E046F10D00001020EF86F8C
:10212A000401056BC80E046F0401080E016F280E26
:10213A00026F040E036FC80E006F6D981200000143
:10214A00F86B0DD8880E006F0401046B1200FCC0F6
:10215A00E9FFFDC0EAFFEF6E0001D0EF10F00401C5
:10216A00080E016F200E026F040E036F1200D9CF02
:10217A00E9FFDACFEAFFEE50ED101200D9CFE6FF01
:10218A00E1CFD9FF020EE1261200D9CFE1FFE552D5
:10219A00E7CFD9FF1200FC2B000EFD23FA2BFB23FD
:1021AA00DF06010E120004012051600BE842E842EA
:1021BA00E842E842E842000901E012002151070A18
:1021CA0040E00B0A3EE0070A33E0010A23E00B0A6B
:1021DA001FE0020A1DE0030A19E0080A10E0010ADA
:1021EA000CE00F0A08E0030A01E0120012D902010A
:1021FA00040EF56F120027EF11F05EEF11F009D906
:10220A000001F70EFA6F020EFB6F0CD079EF11F096
:10221A00ABEF11F002D90001FA6FFB6BF80EFA2747
:10222A00020EFB230201F6930001010EFE6F12005B
:10223A00F4D8EA6AF80FE96E020EEA2222C4EFFF26
:10224A0012001200800E0401205D32E12351030ABC
:10225A001FE0010A0AE0030A29E1DBD80001160E91
:10226A00FA6F270EFB6F120E1ED0ADD8D70EF626C8
:10227A00270EBBD8020E0001F76AFA25F66EFB514B
:10228A00F7220900F5CFFEF00A00F5CFFFF00ED0D5
:10229A009AD8DB0EF626270EA8D8FAC0F6FFFBC09E
:1022AA00F7FF0800F5500001FE6FFF6B0201F6838D
:1022BA001200AFD80F0EE66E710EE66E0F0E9DD8A5
:1022CA00010EE66EF80EE66E020E97D822C4F7F2F9
:1022DA000401225104E10201050EF56F1200020108
:1022EA00060EF56F66EF0EF00401286B296B0401E8
:1022FA0020511F0B020A0FE0030A0BE0010A18E142
:10230A0088D8040128810201F6A112D00401288389
:10231A000FD07FD80DD04BD801E0010E5DD8FCC09C
:10232A00E9FFEA6EEF50040B03E00401010E286F87
:10233A000001F9050AE10001280EFA6F040EFB6F8D
:10234A000201F6930001020EFE6F1200040122053B
:10235A000EE120511F0B00090AE15BD8030E0401AC
:10236A00215D03E10201F68102D00201F691040126
:10237A0022511CE120511F0B020818E124510F0BB6
:10238A00000914E014D801E0010E26D8030E040156
:10239A00215D04E1840E38D8EF6E120024AF03D019
:1023AA0033D8EF6A1200880E2FD8EF6E120035D894
:1023BA000F0B080DF350156A000F146E040E152248
:1023CA002451800B120025D804012251F66EF76AB7
:1023DA00D890F636F7361200040DF3500001142493
:1023EA00FC6F000E1520FD6F1200F7220900F5CFD1
:1023FA00FAF00A00F5CFFBF01200E66EBCEC12F020
:10240A00E552E552E5521200FCC0E9FFFDC0EAFFC1
:10241A0012000001010EF96F1200FBDF04012451C2
:10242A0012006DA60CD80201F50508E16DBA06D0B6
:10243A00686A696A69806988020EF56F12006D6AB6
:10244A00696A6D860201010EF56F12006D6A696A8A
:10245A000201F56B12002BEF12F00201F55101E1B6
:10246A0012006850040B04E06950040B01E03CD8E8
:10247A006DB212006850010B04E06950010B01E0D3
:10248A0054D86850100B04E06950100B01E024D8AE
:10249A006850400B04E06950400B01E03BD868509B
:1024AA00200B04E06950200B01E036D86850020B7B
:1024BA0004E06950020B01E036D8030E0201F55D13
:1024CA0001E212006850080B06E06950080B03E0AD
:1024DA0090EC0FF068961200698468986D82A19A50
:1024EA00A08A0300A09A12006D926994689412005F
:1024FA000201F6A10ED0F8DF6D840201080EF96F11
:10250A00070EFA6FF907000EFA5BF951FA11FAE1B0
:10251A006D941200689C120070A003D0A4EC10F015
:10252A007090689A1200689212006A6A686A9F0E2E
:10253A006B6E7B0E696E6E6A0F0EE66E710EE66E3C
:10254A000F0EE66E14D8E552E552E552160E706E7D
:10255A0068A602D06896FCD76D98A4EC10F0020128
:10256A00F6910201F76B0201030EF56F1200D9CF43
:10257A00E6FFE1CFD9FFFD0EDBCFE9FFFE0EDBCF91
:10258A00EAFFFC0EDB5004E0EE6AFC0EDB06F9D72C
:10259A00E552E7CFD9FF1200DACFE4FFE9CFE4FF33
:1025AA00EACFE4FFE6529EA45AD00001DDB121D061
:1025BA00BD6A060EBD6E9E94DD81BF501E6E1D6AF9
:1025CA00BE5000011D24EA6F000E1E20EB6F0001B1
:1025DA00DE6BDF6B9EA009D09E900001000ED880B2
:1025EA00EA55010EEB5501E282D80001E06BE16B7E
:1025FA0041D09E94DD83BF501D6E1E6A1E6E1D6AF9
:10260A00BE5000011D24E66F000E1E20E76FDEC0DB
:10261A00E8F0DFC0E9F09EA014D09E9068D80001CF
:10262A00E65D010EE75904E20001E82B000EE923FA
:10263A004CD807E353D804E30001DD85F29C01D0AE
:10264A0032D80001E02B000EE1230001ED51000118
:10265A00E05D0001EE510001E1590CE306D09E90C5
:10266A0046D833D807E33AD804E30001DD85F29C63
:10267A0001D019D8E552E5CFEAFFE5CFE9FFE5CF6A
:10268A00DAFF1100D8CFE4FFE0CFE4FFE46EDACF3F
:10269A00E4FFE652E552E5CFDAFFE550E5CFE0FF89
:1026AA00E5CFD8FF10000001EC5126D8EECFE2F0BA
:1026BA00EDCFE3F0EC29EC6FE8501ED8EECFE4F052
:1026CA00EDCFE5F0EC29EC6F12000001E2510001B8
:1026DA00DE5D0001E3510001DF5912000001E451FF
:1026EA000001E05D0001E5510001E159120000011D
:1026FA00DE2B000EDF231200E96EEA6AD890E93673
:10270A00EA36600EE926000EEA22120012010002E1
:10271A0002000008DB045B0000000102000109025C
:10272A004300020100803209040000010202010094
:10273A0005240010010424020205240600010524D0
:10274A000100010705820308000209040100020AC8
:10275A00000000070503024000000705830240004D
:10276A000004030904340348006F006D0065006328
:10277A000069006E0065006D0061002D0066007240
:10278A00002E0063006F006D002000200020002052
:10279A00002000200020002000340343006F006C5A
:1027AA00006F00720069006D0065007400720065B8
:1027BA00002000480043004600520020002000206C
:1027CA0000200020002000200020002000282728C8
:1027DA00276B276F27A327281CFF2A0EF66E080EE1
:1027EA00F76E000EF86E02010900F550F06F09004D
:1027FA00F550F16F03E1F06701D03DD00900F550C3
:10280A00EB6F0900F550EC6F0900F550ED6F090008
:10281A000900F550E96E0900F550EA6E0900090051
:10282A000900F550EE6F0900F550EF6F0900090035
:10283A00F6CFF2F2F7CFF3F2F8CFF4F2EBC2F6FFEB
:10284A00ECC2F7FFEDC2F8FF0201EE5302E1EF53CB
:10285A0007E00900F550EE6EEE07F8E2EF07F9D748
:10286A00F2C2F6FFF3C2F7FFF4C2F8FF0201F00763
:10287A00000EF15BBFD7120006C012F006500B0221
:10288A00F4CF05F0F3CF04F007500C02F4CF07F0B1
:10289A00F3CF06F00B02F3500526F4500622E86A3D
:1028AA00072212500C02F3500526F4500622E86A59
:1028BA000722000C04D80FD82BEC04F0FCD70F0E1B
:1028CA00C112140E6F6E0201F56B0201F66B020162
:1028DA00F76B1CEF04F016EC12F06FBE02D032EC6C
:1028EA0012F000EF0FF0036A026A100EE76ED8903A
:1028FA0006360736023603360B50025C0C50035874
:10290A0005E30B50025E0C50035A062AE72EF0D755
:10291A001200036A080EE76ED890073603360C5089
:10292A00035C02E3036E072AE72EF7D7120013EEC1
:10293A0000F023EE00F0F86A0F9CF2EC13F05FEC63
:10294A0014F0FDD7120076352E31300D0A000D0A2B
:10295A000030313230303400FCFF5C008000B700B8
:10296A0010006E0108003803040001050000FE7F14
:10297A002E0040005C000800B70004009C01020021
:10298A0080020000FF3F170020002E0004005C00B8
:10299A000200CE00020040010000FF3F17002000A5
:1029AA002E0004005C000200CE000200400100007C
:1029BA00FF1F0C001000170002002E000200670023
:1029CA000200A0000000909192939495969798998E
:1029DA009A9B9C9DFFFFFFFFFFFFFFFFFFFFFFFF8B
:020000040020DA
:020000040030CA
:0E000000200E291E008180000FC00FA00F40AF
:0200000400F00A
:00000001FF
